:1000000012C0189518951895189518951DC5A6C471
:100010001895189518951895189518951895189578
:100020001895189518958FE58DBFC0E4E8E34E2E1E
:1000300084E08EBFD4E0F4E05F2EEEEFF3E0A0E6C4
:10004000B0E088278D933197E9F79FD86624A8956B
:1000500084B7877F84BF8CE181BD84E081BD81B599
:10006000886181BD877F81BD90D88AE090E0F3D818
:100070008CD878D8ECE8F0E088E4C4D858E0C8958B
:10008000802DB0D831965A95D1F704C000000000F9
:100090000000001FECEAF0E080E5B4D858E0C89515
:1000A000802DA0D831965A95D1F704C000000000E9
:1000B00000001F1FECECF0E088E5A4D858E0C895DC
:1000C000802D90D831965A95D1F704C000000000D9
:1000D000001F1F1FECEEF0E080E694D858E0C895B2
:1000E000802D80D831965A95D1F704C000000000C9
:1000F0001F1F1F1FECE0F1E088E684D858E0C89588
:10010000802D70D831965A95D1F704C00000001F99
:100110001F1F1F1FECE2F1E080E774D858E0C8957C
:10012000802D60D831965A95D1F704C000001F1F6A
:100130001F1F1F1FECE4F1E088E764D858E0C89562
:10014000802D50D831965A95D1F704C0001F1F1F3B
:100150001F1F1F1F07D88CE055D882E086B980E4A6
:1001600087B9379A80E08FBD81E08EBD81E292E051
:1001700090934B0080934A0080EE9EE2909349005A
:100180008093480089B7846089BF81E08EBD7894F0
:100190008BB78F7B8BBF8BB78F778BBF80E08093C4
:1001A0006000009160000F3110F009F027C0EAE60E
:1001B000F0E1A0E6B0E08C919927A0E6B0E0AD9028
:1001C000BB24AEE6B1E0AA0CBB1CAA0DBB1DC0D976
:1001D000EAEAF0E1A0E6B0E08C919927A0E6B0E071
:1001E000AD90BB24AEE2B1E0AA0DBB1DB6D9A0E62E
:1001F000B0E08C918F5F8C9308F4D3CFEAE6F0E106
:1002000080E090E0AEEAB1E0A3D9EAE6F0E181E077
:1002100090E0A0EBB1E09CD9EAE6F0E182E090E06A
:10022000A2EBB1E095D9EAE6F0E183E090E0A4EB3F
:10023000B1E08ED9EAE6F0E184E090E0A6EBB1E02F
:1002400087D9EAE6F0E185E090E0A8EBB1E080D95B
:10025000EAE6F0E186E090E0AAEBB1E079D9EAE6DF
:10026000F0E187E090E0ACEBB1E072D981B5886055
:1002700081BDA895D2D30027A9E6B0E08C9187FB79
:100280000EF401E041E0041709F001C0F4CF4FD3B0
:1002900028D13CD2F5D410D039D235D40027A9E6E4
:1002A000B0E08C9187FB0EF401E041E0041709F007
:1002B00001C0F4CFB8D5DDCF80E090E0A2EFB1E08F
:1002C0008D939C9381E080936000009160000032E8
:1002D00010F009F039C0A0E6B0E0AD90BB24ACEA64
:1002E000B0E0AA0CBB1CAA0DBB1D0D911C9115956D
:1002F000079515950795A0E6B0E0AD90BB24ACEA54
:10030000B0E0AA0CBB1CAA0DBB1D0D931C93A2EF61
:10031000B1E00D911C91A0E6B0E0AD90BB24ACEA39
:10032000B0E0AA0CBB1CAA0DBB1D4D915C91040F43
:10033000151FA2EFB1E00D931C93A0E6B0E08C91E5
:100340008F5F8C9308F4C1CFA2EFB1E00D911C91A7
:100350001595079515950795159507951595079585
:1003600015950795A2EFB1E00D931C9381E0809362
:10037000600000916000003210F009F0B1C0A0E60A
:10038000B0E0AD90BB24ACEAB0E0AA0CBB1CAA0D57
:10039000BB1D0D911C91A2EFB1E04D915C91041B2E
:1003A000150BA0E6B0E0AD90BB24ACE6B0E0AA0C23
:1003B000BB1CAA0DBB1D0D931C93A0E6B0E0AD9035
:1003C000BB24ACE6B0E0AA0CBB1CAA0DBB1D0D9172
:1003D0001C91A0E6B0E0AD90BB24ADE2B1E0AA0D67
:1003E000BB1D4D91552746D7A0E6B0E0AD90BB248C
:1003F000ACE6B0E0AA0CBB1CAA0DBB1D0D931C9370
:10040000A0E6B0E0AD90BB24ACE6B0E0AA0CBB1C0B
:10041000AA0DBB1D0D911C91159507951595079576
:1004200015950795159507951595079515950795B4
:100430001595079515950795A0E6B0E0AD90BB24FE
:10044000ACE6B0E0AA0CBB1CAA0DBB1D0D931C931F
:10045000A0E6B0E0AD90BB24ACE6B0E0AA0CBB1CBB
:10046000AA0DBB1D0D911C910F3750E0150714F01C
:1004700009F001C00EC08FE790E0A0E6B0E0AD90BB
:10048000BB24ACE6B0E0AA0CBB1CAA0DBB1D8D932F
:100490009C93A0E6B0E0AD90BB24ACE6B0E0AA0C23
:1004A000BB1CAA0DBB1D0D911C9101385FEF1507F8
:1004B0000CF401C00EC081E89FEFA0E6B0E0AD9063
:1004C000BB24ACE6B0E0AA0CBB1CAA0DBB1D8D93EF
:1004D0009C93A0E6B0E08C918F5F8C9308F449CF99
:1004E000089580E090E0A2EFB1E08D939C9381E0CD
:1004F0008093600000916000003210F009F039C074
:10050000A0E6B0E0AD90BB24ACEEB0E0AA0CBB1C02
:10051000AA0DBB1D0D911C91159507951595079575
:10052000A0E6B0E0AD90BB24ACEEB0E0AA0CBB1CE2
:10053000AA0DBB1D0D931C93A2EFB1E00D911C9170
:10054000A0E6B0E0AD90BB24ACEEB0E0AA0CBB1CC2
:10055000AA0DBB1D4D915C91040F151FA2EFB1E0D8
:100560000D931C93A0E6B0E08C918F5F8C9308F400
:10057000C1CFA2EFB1E00D911C911595079515958E
:100580000795159507951595079515950795A2EF6C
:10059000B1E00D931C9381E08093600000916000B6
:1005A000003210F009F0B1C0A0E6B0E0AD90BB247D
:1005B000ACEEB0E0AA0CBB1CAA0DBB1D0D911C91AA
:1005C000A2EFB1E04D915C91041B150BA0E6B0E0E9
:1005D000AD90BB24ACE6B0E0AA0CBB1CAA0DBB1DC1
:1005E0000D931C93A0E6B0E0AD90BB24ACE6B0E068
:1005F000AA0CBB1CAA0DBB1D0D911C91A0E6B0E07E
:10060000AD90BB24ADE2B1E0AA0DBB1D4D915527C5
:1006100031D6A0E6B0E0AD90BB24ACE6B0E0AA0CC9
:10062000BB1CAA0DBB1D0D931C93A0E6B0E0AD90C2
:10063000BB24ACE6B0E0AA0CBB1CAA0DBB1D0D91FF
:100640001C91159507951595079515950795159581
:100650000795159507951595079515950795159582
:100660000795A0E6B0E0AD90BB24ACE6B0E0AA0CE4
:10067000BB1CAA0DBB1D0D931C93A0E6B0E0AD9072
:10068000BB24ACE6B0E0AA0CBB1CAA0DBB1D0D91AF
:100690001C910F3750E0150714F009F001C00EC08F
:1006A0008FE790E0A0E6B0E0AD90BB24ACE6B0E010
:1006B000AA0CBB1CAA0DBB1D8D939C93A0E6B0E0B9
:1006C000AD90BB24ACE6B0E0AA0CBB1CAA0DBB1DD0
:1006D0000D911C9101385FEF15070CF401C00EC09D
:1006E00081E89FEFA0E6B0E0AD90BB24ACE6B0E0BF
:1006F000AA0CBB1CAA0DBB1D8D939C93A0E6B0E079
:100700008C918F5F8C9308F449CF089581E080939A
:100710006000009160000F3010F009F007C180E028
:1007200090E0AAE6B0E08D939C9380E090E0ACE688
:10073000B0E08D939C9380E0809361000091610014
:100740000F3110F009F098C00091610040916000F5
:10075000049F802CA8E0B0E08C918F718C93A8E06E
:10076000B0E0AD90BB24AEE6B1E0AA0CBB1CAA0D74
:10077000BB1D0D911C91A1E6B0E0AD90BB24AEE68F
:10078000B0E0AA0CBB1CAA0DBB1D4D915C9172D5AB
:10079000A2E6B0E00D931C93A8E0B0E0AD90BB24BE
:1007A000ACE7B1E0AA0CBB1CAA0DBB1D0D911C91BE
:1007B000A1E6B0E0AD90BB24AEE6B0E0AA0CBB1C55
:1007C000AA0DBB1D4D915C9155D5A4E6B0E00D93EB
:1007D0001C93A2E6B0E00D911C9115950795159517
:1007E00007951595079515950795159507951595F1
:1007F00007951595079515950795A2E6B0E00D9319
:100800001C93A4E6B0E00D911C91159507951595E4
:1008100007951595079515950795159507951595C0
:1008200007951595079515950795A4E6B0E00D93E6
:100830001C93AAE6B0E00D911C91A4E6B0E04D91A6
:100840005C91040F151FAAE6B0E00D931C93ACE673
:10085000B0E00D911C91A2E6B0E04D915C91041BBB
:10086000150BACE6B0E00D931C93A1E6B0E08C91C3
:100870008F5F8C9308F462CFAAE6B0E00D911C91D3
:10088000159507951595079515950795AAE6B0E076
:100890000D931C93ACE6B0E00D911C911595079556
:1008A0001595079515950795ACE6B0E00D931C934B
:1008B000AAE6B0E00D911C91AAE6B0E04D915C91E2
:1008C000D9D4A4E6B0E00D931C93ACE6B0E00D9152
:1008D0001C91ACE6B0E04D915C91CCD4A2E6B0E0C6
:1008E0000D931C93A4E6B0E00D911C91A2E6B0E03C
:1008F0004D915C91040F151FA4E6B0E00D931C937D
:10090000A4E6B0E033D6A0E6B0E0AD90BB24AEE400
:10091000B1E0AA0CBB1CAA0DBB1D4D935C93A0E6D5
:10092000B0E08C918F5F8C9308F4F3CE089587E04C
:1009300086B980E487B9379A80E090E090934D00C3
:1009400080934C0089B7886089BF80E080936800FD
:100950008091690080688093690008950F921F92CA
:100960002F923F924F925F927F92AF92BF920F93DE
:100970001F932F933F934F935F936F937F938F9327
:100980009F93AF93BF93CF93DF93EF93FF938FB773
:100990008F9380E090E090934D0080934C00A8E608
:1009A000B0E08C918F5F8C9381E4806487B96CD4C4
:1009B000A8E6B0E0AD90BB24ACEEB0E0AA0CBB1C46
:1009C000AA0DBB1D8D939C9300916800003209F025
:1009D00008C089B7877F89BF809169008F7780932E
:1009E00069008F918FBFFF91EF91DF91CF91BF9100
:1009F000AF919F918F917F916F915F914F913F91B7
:100A00002F911F910F91BF90AF907F905F904F906B
:100A10003F902F901F900F90189581E086B980E449
:100A200087B9379A80E090E090934D0080934C0016
:100A300089B7806189BF80E08093680080916900F8
:100A400080688093690008950F921F922F923F92C1
:100A50004F925F927F92AF92BF920F931F932F930B
:100A60003F934F935F936F937F938F939F93AF9336
:100A7000BF93CF93DF93EF93FF938FB78F9380E074
:100A800090E090934D0080934C00A8E6B0E08C91EC
:100A90008F5F8C9380E4806487B9F6D3A8E6B0E0DA
:100AA000AD90BB24ACEAB0E0AA0CBB1CAA0DBB1DE8
:100AB0008D939C9300916800003209F008C089B7BB
:100AC0008F7E89BF809169008F77809369008F91B5
:100AD0008FBFFF91EF91DF91CF91BF91AF919F9128
:100AE0008F917F916F915F914F913F912F911F91C6
:100AF0000F91BF90AF907F905F904F903F902F905D
:100B00001F900F901895A2E5B1E08D919C91A6E6FB
:100B1000B0E08D939C93809166008093CA01A4E518
:100B2000B1E08D919C91A6E6B0E08D939C9380916D
:100B300066008093CB01A6E5B1E08D919C91A6E67D
:100B4000B0E08D939C93809166008093CC01A8E5E2
:100B5000B1E08D919C91A6E6B0E08D939C9380913D
:100B600066008093CD01AAE5B1E08D919C91A6E647
:100B7000B0E08D939C93809166008093CE01ACE5AC
:100B8000B1E08D919C91A6E6B0E08D939C9380910D
:100B900066008093CF01AEE5B1E08D919C91A6E611
:100BA000B0E08D939C93809166008093D001A0E685
:100BB000B1E08D919C91A6E6B0E08D939C938091DD
:100BC00066008093D101A2E6B1E08D919C91A6E6EA
:100BD000B0E08D939C93809166008093D201A4E64F
:100BE000B1E08D919C91A6E6B0E08D939C938091AD
:100BF00066008093D301A6E6B1E08D919C91A6E6B4
:100C0000B0E08D939C93A6E6B0E04D915C91A8E690
:100C1000B1E00D911C910417150714F009F001C003
:100C200008C0A8E6B1E08D919C91A6E6B0E08D9356
:100C30009C93809166008093D401AAE6B1E08D91E7
:100C40009C91A6E6B0E08D939C93A6E6B0E04D9112
:100C50005C91ACE6B1E00D911C910417150714F0FE
:100C600009F001C008C0ACE6B1E08D919C91A6E608
:100C7000B0E08D939C93809166008093D501089598
:100C8000A0E5B1E08D919C91A6E6B0E08D939C9398
:100C9000809166008093BE01A2E5B1E08D919C91A8
:100CA000A6E6B0E08D939C93809166008093BF018F
:100CB000A4E5B1E08D919C91A6E6B0E08D939C9364
:100CC000809166008093C001A6E5B1E08D919C9172
:100CD000A6E6B0E08D939C93809166008093C1015D
:100CE000A8E5B1E08D919C91A6E6B0E08D939C9330
:100CF000809166008093C201AAE5B1E08D919C913C
:100D0000A6E6B0E08D939C93809166008093C3012A
:100D1000ACE5B1E08D919C91A6E6B0E08D939C93FB
:100D2000809166008093C401AEE5B1E08D919C9105
:100D3000A6E6B0E08D939C93809166008093C501F8
:100D4000A0E6B1E08D919C91A6E6B0E08D939C93D6
:100D5000809166008093C601A2E6B1E08D919C91DE
:100D6000A6E6B0E08D939C93A6E6B0E04D915C9131
:100D7000A4E6B1E00D911C910417150714F009F0D9
:100D800001C008C0A4E6B1E08D919C91A6E6B0E058
:100D90008D939C93809166008093C701A6E6B1E095
:100DA0008D919C91A6E6B0E08D939C93A6E6B0E071
:100DB0004D915C91A8E6B1E00D911C9104171507C7
:100DC00014F009F001C008C0A8E6B1E08D919C9133
:100DD000A6E6B0E08D939C93809166008093C80155
:100DE000AAE6B1E08D919C91A6E6B0E08D939C932C
:100DF000A6E6B0E04D915C91ACE6B1E00D911C919E
:100E00000417150714F009F001C008C0ACE6B1E002
:100E10008D919C91A6E6B0E08D939C9380916600A5
:100E20008093C901089581E0809360000091600083
:100E3000083110F009F0FAC0EAEBF6E16DD3E0E614
:100E4000F0E0A190BB24EDEBF1E0EA0DFB1DD080BA
:100E5000EE24FF24002783D2CBD2EDE0F0E0AEEE0B
:100E6000B1E07ED3EEEEF1E01CD4EDE0F0E0AEEECA
:100E7000B1E076D3EEEEF1E053D2EEEBF6E143D300
:100E8000B7D2EDE0F0E0AEEEB1E06AD3E2ECF6E12D
:100E900043D3EEEEF1E03FD2E4D2EDE0F0E0FDD15D
:100EA000A4E6B0E0EE0C000FE794DD92EC92A4E62D
:100EB000B0E00D911C91003050E015070CF401C01A
:100EC00006C080E090E0A4E6B0E08D939C93A4E699
:100ED000B0E00D911C91003150E0150714F009F0BD
:100EE00001C006C080E190E0A4E6B0E08D939C9341
:100EF00080916400A0E6B0E0AD90BB24ADEBB1E022
:100F0000AA0DBB1D8C93A0E6B0E0AD90BB24A5ED6F
:100F1000B1E0AA0DBB1D4C91A0E6B0E0AD90BB24A2
:100F2000ADEBB1E0AA0DBB1D0C91041710F009F058
:100F300001C013C0A0E6B0E0AD90BB24ADEBB1E0C2
:100F4000AA0DBB1D8C91A0E6B0E0AD90BB24A5ED31
:100F5000B1E0AA0DBB1D8C9338C0A0E6B0E0AD9007
:100F6000BB24A5E2B2E0AA0DBB1D0C91013009F033
:100F700021C0A0E6B0E0AD90BB24A5EDB1E0AA0D84
:100F8000BB1D0C91003010F009F001C009C0A0E6B3
:100F9000B0E0AD90BB24A5EDB1E0AA0DBB1DB5D06E
:100FA00080E0A0E6B0E0AD90BB24A5E2B2E0AA0DDF
:100FB000BB1D8C93A0E6B0E0AD90BB24A5E2B2E0EF
:100FC000AA0DBB1D8C918F5F8C93E6E4F0E1A0E647
:100FD000B0E0AD90BB24A5EDB1E0AA0DBB1D8C9196
:100FE0009927A0E6B0E0AD90BB24A3EFB1E0AA0D35
:100FF000BB1DB3D2E8E5F0E1A0E6B0E0AD90BB24C4
:10100000A5EDB1E0AA0DBB1D8C919927A0E6B0E03B
:10101000AD90BB24ACE0B2E0AA0DBB1D9ED2A0E611
:10102000B0E08C918F5F8C9308F400CF8FE711E0D4
:10103000AAD0A4EFB1E090D08FEB11E0A4D0ADE046
:10104000B2E08AD0089520202020202020202001F6
:10105000020304050607FF0020010203040506073A
:10106000FFFFFFFFFFFFFFFFFF00000032006200F5
:101070008E00B500D500ED00FB00FF00FB00ED0089
:10108000D500B5008E00620032000000CEFF9EFF4A
:1010900072FF4BFF2BFF13FF05FF01FF05FF13FF3F
:1010A0002BFF4BFF72FF9EFFCEFF00030A17283C69
:1010B000546D86A0B8CEE1F0FAFFFFFAF0E1CEB8A9
:1010C000A0866D543C28170A030014171E2A394CB9
:1010D000617890A8BED2E4F1FBFFFFFBF1E4D2BE41
:1010E000A89078614C392A1E17140001040A121FB7
:1010F00030455E7A97B5D0E6F6FFFFF6E6D0B597B5
:101100007A5E45301F120A0401008C9181508C9345
:10111000089504D0AFD000FC0CD008950024E894CA
:1011200057FF02C009D0689400F80BD010F80124D2
:10113000089502D009D00895509540954F5F5F4FB4
:101140000895E89417FF0895009510950F5F1F4FBD
:1011500068940895A0E2B4E08D91882311F042D004
:10116000FBCF089581E04ED0E4EBFBE038D080E87F
:1011700049C08FE7213039F08FEB223021F08FE822
:10118000233009F08FEC810F3DC0882782BB8FEFA1
:1011900081BBECE1FEE423D080E382BB939A0000A4
:1011A00000009398E4E8F3E11AD0939A000000005D
:1011B0009398E0E6F0E013D0939A00000000939833
:1011C000E0E6F0E00CD080E282BB939A00000000E1
:1011D000939888E217D08EE015D086E013C031973F
:1011E000F1F7089519D090EF982392BB919A05D00A
:1011F0009FE09823929592BB919A939A00000000E9
:101200009398089509D090EF982392BBF6DF8295CA
:1012100090EF982392BBF1CF9FE091BB992792BBAF
:10122000929A939A0000000090B3939800000000F7
:10123000939A00000000939897FDEECF92989FEF4D
:1012400091BB08953197F1F70895689462F8089575
:10125000E89462F80895EF93FF93EE27E82BE92BCB
:1012600031F0E0E7F7E13197F1F70197D1F7FF911E
:10127000EF9108950F92B801469F8001479F100D8E
:10128000569F100D0F900895369A3699FECF369AD4
:101290003699FECF84B195B108953DD09927112795
:1012A0008F2D880F80E8F82A802F881F08F41FEF01
:1012B00041F08F57082F07FD04C0003240F08FEF38
:1012C00001C08827982FD82EE82EF82E09C08FE16C
:1012D000801B082FF694E794D79497950A95D1F739
:1012E000112351F09095D094E094F09481E0980F00
:1012F0008827D81EE81EF81E0F2DFE2CED2CD92EA7
:101300000895D094E094F09491E0D90E9927E91EC5
:10131000F91E10950895D190E190F19001910895F2
:1013200021913191419151910895102F90E8FF0C36
:10133000001F0927990FF7941078652F90E8440F44
:10134000551F5927990F4795607800380895FF0C6D
:1013500090E89027110F9795F794092F0895102F73
:10136000BD2CDE2CEF2CF02E11234AF4B094D09437
:10137000E094F0949FEFB91AD90AE90AF90A0EE14C
:10138000FF2039F4FE2CED2CDB2CBB240850C2F7D7
:1013900029C032F00A95BB0CDD1CEE1CFF1CF9CFF6
:1013A00001D0D5CFB7FE089590E8B91611F4D0FE5C
:1013B00008959FEFD91AE90AF90A09F403950895E7
:1013C000DD92ED92FD920C930895502F2D2D3E2D20
:1013D0004F2D612F08959FE7092FF92A9FEFD92EEE
:1013E000E92E0895DD24EE24FF2400271127089517
:1013F0009CDFC1F35038B1F31627005850580894B9
:10140000051F12F418F4E7CF08F0ECCF0AD0FF2044
:101410002AF0BB0CDD1CEE1CFF1C99CF0F5FDBF22A
:1014200096CF9F929924AA24BB24992788E1990CEE
:10143000AA1CBB1CDD1CEE1CFF1C30F4920EA31E6C
:10144000B41ED91EE91EF91E8A9589F79F9008954A
:101450000AF045D07CCF5FE322273327442701C021
:101460005FDF63DF5038B1F3003899F3902F951B9D
:101470008BF312F434D0FACF983118F022273327A7
:101480004427983028F0232F342F44279850F9CF41
:10149000992329F04695379527959A95D9F7912F55
:1014A000962742F014D0B0F6F794E794D7940F5FE4
:1014B0008BF691CF10D051F008F423DFFF2052F2C9
:1014C000DD0CEE1CFF1C0150CBF785CF8BCFD20E6D
:1014D000E31EF41E0895D21AE30AF40A0895DF9277
:1014E000EF92FF920F931F93D22EE32EF42E052F2F
:1014F000162F6F915F914F913F912F910895C8954D
:10150000319600200895FBDFD02CF9DFE02CF7DFC7
:10151000F02CF5DF002D0895F2DF202DF0DF302DC7
:10152000EEDF402DECDF502D089500240D280E280D
:101530000F28002A0020089591E005C092E003C022
:1015400094E001C098E0DBDF0D929A95E1F70895F1
:10155000880F991FE80FF91FF1CFE80FF91FECCFA3
:1015600094E081918D939A95E1F708950D911C91E6
:1015700011231AF425C00D911C9199272227332796
:101580004427552789E0440F551F000F111F221FC4
:10159000331F000F111F221F331F642F752F660F7B
:1015A000771F63952617370720F0261B370B4395C7
:1015B000591F8A9541F756954795491F591F089518
:1015C0004427552708950ECFA6DE0023E2F3ADDFB2
:1015D00019F401DF0068089585E050D0FF0C001F6A
:1015E00004830FE70695F79463D050683ADFE8DE8E
:1015F000139721E438E743ED5BEBFADE27E831EDA2
:1016000043E15DE337D02EE03CE343EC5DEB32D0C9
:1016100022E83DEA4BE25EE32DD02CEE32E846E7CD
:101620005EEB28D020E931EE49EA5EE323D020E8E2
:101630003FEE4FEF5EEB1ED024EC3FEF4FE75FE352
:1016400019D0BEDE139784818F5799F02AF4D82ED3
:101650000FEFE02EF02E04C0D82EEE24FF2400273A
:101660007EDE28E132E741E35FE3C2DE59DE3497F4
:10167000F8DE11C0F6DE54DE3497BACE0FB6F89419
:101680004A925A92E42DF52DA42DB52D480E8827A7
:10169000581E0FBE08950FB6F894599049900FBE8A
:1016A000089539DE92DF29ED3BE54EED5EE3A0CEF5
:1016B0005FE340E8332722270895CDCCCC3D0000DE
:0616C000A0410000000043
:00000001FF
